:100000000C94B9020C9400030C9400030C940003AC
:100010000C9400030C9400030C9400030C94000354
:100020000C9400030C9400030C94170C0C94E90C32
:100030000C9400030C9400030C9400030C94000334
:100040000C9400030C945D210C9400030C940003A9
:100050000C9400030C94EF1A0C9400030C9400030E
:100060000C9400030C9400030C9400030C94000304
:100070000C9400030C9400030C9400030C940003F4
:100080000C9400030C9400030C9400030C940003E4
:100090000C9400030C9400030C9400030C940003D4
:1000A0000C9400030C9400030C940003560D780D7F
:1000B0006B0E780D6B0EBD0DE00D6B0E350E480E00
:1000C0003211321161116111A411DE11EB13EB1326
:1000D000F711EB13EC12EC12BF13EB13EB13D61367
:1000E0000000F0A12E002B002900E1003581000066
:1000F0001E00140004001D713400E2001F001A00ED
:1001000016001B00E1044C00200008000700060058
:1001100050002A0021001500090019004F004D0071
:10012000220017000A00050000006574E300015476
:100130000000007F00004A004F00035400000077D9
:100140000000E20023001C000B00110000002971D8
:10015000240018000D00100052004B0025000C0078
:100160000E00360051002C00260012000F00370050
:100170002F002800270013003382387130004E0012
:100180002D0031003400E500C10000000100010035
:1001900001000100010000003A001E0220022202BC
:1001A000010001003B001F022102230201000100A7
:1001B0003C002F0226022F00010001003D0030020A
:1001C00027023000010001003E00310235003502F7
:1001D000000001000100010000000100000001001A
:1001E0000100010000000100000001003F0052007A
:1001F00051002402000001004000240021001E00E4
:10020000010001004100250022001F00370001000D
:1002100042002600230020002700010043002502A1
:100220002E0231002E0001004400450001000100B3
:1002300001000000010001000100010001000000B8
:1002400001000100010001000100010001000100A6
:10025000F20001000100F5000100F000F1000100D2
:10026000F400F40001000100F3000100F5000100BA
:100270000100010001000100000001000100010077
:100280000000010000000100010001000000010069
:100290000000010001000100F20001000000010067
:1002A00001000100F1000100A900010001000100AE
:1002B000F000AC00AA00B70001000100F300AB00A1
:1002C000A800B600010001000100010001000100CA
:1002D00001000100AE00010001000000000000006C
:1002E000000000000000000000001E0014000400D8
:1002F0000000000000001F001A0016000000190096
:100300000000200008000700000006000000210097
:1003100015000900000000000000220017000A007C
:100320000000C40000000000000000000000000009
:100330000100000000000000000001000000230098
:100340001C000B00000001000000240018000D003C
:1003500001000100000025000C000E00010010004B
:100360000000260012000F0000001100000027000E
:100370001300330000000000010001002F003400D2
:100380000000000016034500720067006F00440083
:100390006F007800200045005A0000001603450059
:1003A000720067006F0044006F0078002000450075
:1003B0005A0000000403090409026D00040100A0B2
:1003C000FA090400000103010100092111010001E3
:1003D000223F000705810308000A09040100010308
:1003E000010200092111010001224D0007058203CD
:1003F00008000A090402000103000000092111019C
:1004000000012236000705830308000A09040300DF
:100410000103000000092111010001223900070534
:1004200084031000011201100100000008EDFE0716
:100430001301000102000105010906A101050719C8
:10044000E029E715002501950875018102050819C5
:100450000129059505750191029501750391010525
:10046000071900297715002501957875018102C0CB
:1004700005010980A101850216010026B7001A01B5
:10048000002AB700751095018100C0050C0901A173
:10049000018503160100269C021A01002A9C0275A0
:1004A0001095018100C005010902A1010901A10007
:1004B0000509190129051500250195057501810218
:1004C0009501750381010501093009311581257FE9
:1004D00095027508810609381581257F95017508F3
:1004E0008106050C0A38021581257F950175088162
:1004F00006C0C005010906A101050719E029E71595
:100500000025019508750181029501750881010595
:100510000819012905950575019102950175039149
:10052000010507190029FF150025FF9506750881AB
:1005300000C00000000000000000000000010204F4
:10054000060A0F17202C3A4A5D71879DB3C7DAE976
:10055000F5FCFFFCF5E9DAC7B39D87715D4A3A2CDB
:1005600020170F0A0604020100000000000000002E
:10057000000011241FBECFEFDAE0DEBFCDBF04B60E
:1005800003FE27C08091ED019091EE01A091EF0153
:10059000B091F0018730904BA740B04BD1F410924E
:1005A000ED011092EE011092EF011092F00114BED5
:1005B00084B7877F84BF0FB6F894A89580916000B8
:1005C000886180936000109260000FBEE0E0FFE35E
:1005D000099511E0A0E0B1E0ECE5F6E402C0059079
:1005E0000D92A433B107D9F721E0A4E3B1E001C033
:1005F0001D92AD3EB207E1F70E945E090C942C23D8
:100600000C94000061110BC0FC018281882321F051
:1006100085EE0E94CC0F03C085EE0E94941080E00E
:1006200090E0089508956091B1017091B2018091B8
:10063000B3019091B4010E941C1A56985E982598B7
:100640002D9826982E9827982F98813019F082306F
:1006500021F00895259A2D9A0895269A2E9A0895A4
:100660000C94130356985E9825982D9826982E98EA
:1006700027982F988FEF90E09093890080938800BF
:1006800090938B0080938A0090938D0080938C00D0
:10069000259A2D9A2FEF80E792E0215080409040DC
:1006A000E1F700C00000269A2E9A2FEF80E792E033
:1006B000215080409040E1F700C00000279A2F9A17
:1006C0002FEF80E792E0215080409040E1F700C09A
:1006D000000025982D982FEF80E792E02150804070
:1006E0009040E1F700C0000026982E982FEF80E799
:1006F00092E0215080409040E1F700C00000279830
:100700002F9856985E9825982D9826982E98279879
:100710002F98089589EA8093800089E08093810072
:1007200024982C983F988AB18F748AB96E98479A0A
:100730008BB1806B8BB9769A0E9432030C941203B2
:1007400080E2809300018091340181110EC00E94EB
:10075000EF0381E0809334012FEF83ED90E321508C
:1007600080409040E1F700C0000080E40E94F50363
:100770008093000181112EC00E941F04809300010C
:10078000811128C00E941F0480930001811122C0A2
:100790008FE30E941F048093000181111BC00E94FF
:1007A000170480E40E94F50380930001811112C0B8
:1007B0008CE00E941F048093000181110BC00E94F5
:1007C0001F0480930001811105C08FE30E941F0464
:1007D000809300010E9417048091000108951092F7
:1007E000B9008AE08093B800089594EA9093BC0021
:1007F0009091BC0097FFFCCF9091B900987F983002
:1008000021F0903111F081E008958093BB0084E8DD
:100810008093BC008091BC0087FFFCCF8091B90021
:10082000887F883111F0803471F780E0089584E981
:100830008093BC008091BC0084FDFCCF0895809320
:10084000BB0084E88093BC008091BC0087FFFCCF94
:100850009091B900987F81E0983209F480E0089582
:1008600084E88093BC008091BC0087FFFCCF80911E
:10087000BB00089580910001811115C080E40E94A1
:10088000F5038093000181110CC082E10E941F04D6
:1008900080930001811105C08FEF0E941F04809397
:1008A00000010E94170484B1807F84B985B1807FE4
:1008B00085B98AB1837F8AB98BB1837F8BB93E9822
:1008C000469808950E94A003809300010E943A0474
:1008D00080B38C7080BB81B3836F81BBE4E4F1E0B3
:1008E000A6E3B1E011921D9281E0E235F807D1F75D
:1008F0000C948A039F92AF92BF92CF92DF92EF92B5
:10090000FF920F931F93CF93DF9380910001882371
:1009100079F0809135018F5F80933501811108C096
:100920000E94A00380930001811102C00E94320343
:1009300086E3E82E81E0F82E8701C0E0D0E0BB24FA
:10094000B39492E0A92ECC24C394D12CC730D10506
:1009500000F580910001811164C080E40E94F503DC
:1009600080930001811112C082E10E941F048093D4
:10097000000181110BC0C6010C2E01C0880F0A9422
:10098000EAF780950E941F04809300010E941704DB
:1009900048C0CA30A1F028F4C83059F0C93061F01D
:1009A00005C0CC3089F070F0CD3089F0209A2898BD
:1009B00010C0219A29980DC0229A2A980AC0239A19
:1009C0002B9807C0529A01C0539A5B9802C03E9A76
:1009D0004698E0EAEA95F1F78FB181708B25799915
:1009E00002C032E001C030E0832B7C9902C034E0C9
:1009F00001C030E0832B7D9902C028E001C020E0D7
:100A0000822B7E9902C090E101C090E0892B9FB1BA
:100A10009095991F9927991F9295990F907E892BF0
:100A20000FC08091000181114AC080E40E94F5034B
:100A300080930001882381F1912C0E941704892D55
:100A4000D8019C91981719F08C93A09201010E94F3
:100A50003A0421960F5F1F4FCE30D10509F076CFB3
:100A600080910101882369F18150809301018823DD
:100A700039F0EFE9FFE03197F1F700C0000021C045
:100A8000E4E4F1E0D7018D917D018193B4E4EB16AC
:100A9000B1E0FB06B9F715C083E10E941F04809303
:100AA00000018111C9CF81E40E94F5038093000108
:100AB0008111C2CF0E943004982E9094BECF80E066
:100AC000BFCF0E94300381E0DF91CF911F910F9142
:100AD000FF90EF90DF90CF90BF90AF909F900895E0
:100AE000E82FF0E0EC5BFE4F8081089508958B3B8A
:100AF000910580F4883A910548F5853A9105D8F436
:100B00008430910508F0B2C0019709F06EC081E011
:100B100090E00895803E910508F467C0883E9105F5
:100B200008F4A4C09C01205F31092031310508F090
:100B30005CC090650895853A910509F459C0863ADC
:100B4000910509F058C082E890E40895883A91052B
:100B500009F454C0893A910509F453C08A3A9105C1
:100B600009F452C08B3A910509F451C08C3A9105B1
:100B700009F450C08D3A910509F44FC0803B9105AE
:100B800009F44EC08E3A910509F44DC08F3A910593
:100B900009F44CC0813B910509F44BC0823B91059F
:100BA00009F44AC0833B910509F449C0843B91058F
:100BB00009F448C0853B910509F447C0863B91057F
:100BC00009F446C0873B910509F445C0883B91056F
:100BD00009F444C0893B910509F443C08A3B91055F
:100BE00009F442C080E094E4089580E090E0089524
:100BF00081E890E4089583E890E4089582EE94E417
:100C0000089589EE94E408958AEE94E4089585EBBE
:100C100094E4089586EB94E4089587EB94E40895B2
:100C20008CEC94E408958DEC94E4089583E895E4C5
:100C300008958AE895E4089582E995E4089584E9A1
:100C400095E4089581E296E4089583E296E4089598
:100C500084E296E4089585E296E4089586E296E4B7
:100C6000089587E296E408958AE296E40895089547
:100C700024E5829FC0011124FC0126E0729FE00D53
:100C8000F11D1124E60FF11DEE0FFF1FEC51FF4F78
:100C9000859194910895880F991FFC01E05AF040C6
:100CA000859194910895880F991FFC01E052FF4FA0
:100CB00085919491089524E5829FC0011124FC013F
:100CC00046E0749FE00DF11D1124E60FF11DEE0FBB
:100CD000FF1FEC51FF4F859194919C013A9521158E
:100CE0004FE1340708F425C13F512115304120F46C
:100CF0009F700E94530608959C0130532115304186
:100D000018F49927906C0895811520E5920769F4ED
:100D10000E940D144FEF84E39CE0415080409040CE
:100D2000E1F700C000000C94141B813020E592070D
:100D300031F48091CC0181608093CC0108959C01B5
:100D400030552115304108F05CC0292F33272F7012
:100D5000332721303105E9F4AC0164E0440F551F1D
:100D60006A95E1F744275370BC016370772702C08E
:100D7000220F331F6A95E2F73C68242B352B73E072
:100D8000880F991F7A95E1F780769927822B932B0C
:100D900008952230310529F4982F8827816F906AB1
:100DA000089523303105A1F4AC0133E0440F551F01
:100DB0003A95E1F7407E57708370992721E030E043
:100DC00002C0220F331F8A95E2F7C9019C6816C042
:100DD0002430310531F5AC0123E0440F551F2A952D
:100DE000E1F7407E57708370992721E030E002C020
:100DF000220F331F8A95E2F7C9019A68842B952B3D
:100E000008959C0130572115304118F49F7090626D
:100E100008959C0130582115304118F49F70906A54
:100E20000895803E9105E0F4803C910558F58133AA
:100E3000910509F46FC048F48932910509F463C043
:100E40008A32910509F46DC072C089339105E9F0C9
:100E500082389105D1F08533910509F44DC067C002
:100E6000833E910581F138F4803E9105B9F0823ED0
:100E70009105D9F05CC0863E910561F1873E9105F0
:100E8000A1F155C00E944B0608952091DE0120FD7E
:100E900002C021FF4CC080EE90E049C08091DE018D
:100EA00080FFF9CF89E390E042C08091DE0182FFAC
:100EB0000EC08091DE0184FF03C080E090E037C067
:100EC00083EE90E034C08091DE0182FFF2CF82EEAB
:100ED00090E02DC08091DE0183FF0BC08091DE0188
:100EE00084FDEBCF87EE90E022C08091DE0183FF8E
:100EF000F5CF86EE90E01BC08091DE0185FF07C034
:100F000089E290E014C08091DE0185FFF9CF85E38E
:100F100090E00DC08091DE0186FF07C08AE290E07C
:100F200006C08091DE0186FFF9CF81E390E00E9448
:100F3000770508950895809162010895CF93DF9316
:100F400000D01F92CDB7DEB79C018091E4018430C0
:100F500019F593E099833B832A839093E9008FEFFF
:100F60009091E800815095FD06C095ED9A95F1F7B6
:100F700000008111F5CF8091E80085FF0DC040E0B1
:100F800050E063E070E0CE0101960E940B0A809170
:100F9000E8008E778093E8000F900F900F90DF911C
:100FA000CF910895CF93DF9300D01F92CDB7DEB7D6
:100FB0002091E401243021F522E029839B838A8358
:100FC00083E08093E9008FEF9091E800815095FDD8
:100FD00006C095ED9A95F1F700008111F5CF80914B
:100FE000E80085FF0DC040E050E063E070E0CE0116
:100FF00001960E940B0A8091E8008E778093E800AA
:101000000F900F900F90DF91CF9108959C018091E8
:10101000E4018430F9F482E08093E9009FEF80914D
:10102000E800915085FD06C085ED8A95F1F7000036
:101030009111F5CF8091E80085FF0CC040E050E0B1
:1010400065E070E0C9010E940B0A8091E8008E778C
:101050008093E8000895CF93DF93EC018091E40141
:10106000843009F046C090910C019923D9F09091F9
:101070000D019923B9F08093E9008FEF9091E8007A
:10108000815095FD06C095E19A95F1F70000811118
:10109000F5CF8091E80085FF2CC040E050E060E192
:1010A00070E017C081E08093E9008FEF9091E80035
:1010B000815095FD06C095ED9A95F1F700008111DC
:1010C000F5CF8091E80085FF14C040E050E068E073
:1010D00070E0CE010E940B0A8091E8008E77809329
:1010E000E80080E1FE01A2E5B1E001900D928A9551
:1010F000E1F7DF91CF9108958091E301811109C05B
:101100000E949C0B0E94F90B8091E2008460809306
:10111000E20008951092E301089508950C944A2185
:101120000E94AA1A0E9450210E94A40E0C949A07B1
:1011300042E061EC81E00E94150B42E061EC82E04C
:101140000E94150B42E061EC83E00E94150B42E126
:1011500061EC84E00C94150B8091E601833009F476
:1011600055C030F4813071F0823009F48EC008959A
:101170008A3009F47AC08B3009F460C0893009F0F4
:101180009CC020C08091E501813A09F096C0809111
:10119000E800877F8093E8008091E9019091EA015F
:1011A000892B21F460E182E591E003C060E080E0FA
:1011B00090E070E00E94560A8091E8008B7780935F
:1011C000E80008958091E501813209F076C08091B0
:1011D000E9019091EA01009719F0039709F06DC0B9
:1011E0008091E800877F8093E8008091E80082FD8D
:1011F00005C08091E4018111F8CF5FC08091F100BA
:10120000809362018091E8008B7753C08091E50163
:10121000813A09F052C08091E9019091EA01892B4D
:1012200009F04BC08091E800877F8093E8008091AF
:10123000E80080FFFCCF80910C0136C08091E50171
:101240008132D9F58091E9019091EA01892BA9F5C4
:101250008091E800877F8093E8000E944A0B80918C
:10126000E70180930C010C940D148091E50181320B
:1012700021F58091E800877F8093E8000E944A0B67
:101280008091E8018093630108958091E501813A9E
:10129000A1F48091E800877F8093E8008091E800C6
:1012A00080FFFCCF809163018093F1008091E80082
:1012B0008E778093E8000C944A0B089584B7877F5B
:1012C00084BF0FB6F894A8958091600088618093E0
:1012D0006000109260000FBE90E080E80FB6F894B6
:1012E00080936100909361000FBE0E94F30E0E94F4
:1012F0009C0B0E94F90B8091E20084608093E200D5
:1013000078940E94840E0E94F50E82E091E00E9483
:101310009F0E0E9438218091E401853069F40E947B
:101320006C1A8091E2018823B1F30E94961A8823F7
:1013300091F30E94F509EFCF0E94FB0EECCF292F0D
:10134000332723303105C9F060F42130310581F0B5
:101350002230310509F041C08DE690E028EB33E002
:1013600040C021323105E1F02232310531F135C082
:1013700082E190E025E234E034C099278130910584
:1013800049F028F0029749F5E4E8F3E005C0E4EB02
:10139000F3E002C0ECE9F3E0849190E09F0121C00A
:1013A0006430D8F4E62FF0E0EE0FFF1FEE5DFE4F45
:1013B0002081318189E090E014C0643070F470E0E5
:1013C000FB01EE0FFF1FE65EFE4F20813181FB0126
:1013D000EA5EFE4F808190E004C080E090E020E073
:1013E00030E0FA0131832083089580E189BD82E1F4
:1013F00089BD09B400FEFDCF8091D8008F7D809318
:10140000D8008091E00082608093E0008091E0004D
:1014100081FDFCCF0895CF92DF92EF92FF920F9360
:101420001F93CF93DF93EC018B016A010E94690B3C
:10143000811133C0C114D10439F0F601808191814A
:10144000081B190BC80FD91FE12CF12C0115110530
:1014500019F18091E80085FD16C08091E8008E7733
:101460008093E800C114D10449F0F6018081918194
:10147000E80EF91EF182E08285E00FC00E94690B40
:10148000882321F30AC089918093F100015011094A
:10149000FFEFEF1AFF0ADACF80E0DF91CF911F91C3
:1014A0000F91FF90EF90DF90CF9008952091EB0186
:1014B0003091EC012617370748F06115710539F4B2
:1014C0002091E8002E772093E80001C0B901FC01CB
:1014D00020E06115710579F18091E4018823F1F133
:1014E0008530F1F18091E80083FD3CC08091E800F7
:1014F00082FD2EC08091E80080FFEBCF2091F300A9
:101500008091F20090E0922B6115710551F08830C6
:10151000910538F421912093F100615071090196F1
:10152000F3CF21E0089709F020E08091E8008E7762
:101530008093E800CECF2111CFCF0AC08091E40183
:10154000882361F0853061F08091E80083FD0AC056
:101550008091E80082FFF2CF80E0089582E0089554
:1015600083E0089581E008952091EB013091EC0132
:101570002617370748F06115710539F42091E80006
:101580002E772093E80001C0B901FC0120E061152D
:10159000710591F18091E401882309F440C0853000
:1015A00009F43FC08091E80083FD3DC08091E800D0
:1015B00082FD2FC08091E80080FFE9CF2091F300E9
:1015C0008091F20090E0922B6115710559F08830FE
:1015D000910540F424912093F100319661507109F6
:1015E0000196F2CF21E0089709F020E08091E80011
:1015F0008E778093E800CBCF2111CCCF0AC08091A9
:10160000E401882361F0853061F08091E80083FD7A
:101610000AC08091E80082FFF2CF80E0089582E066
:10162000089583E0089581E00895982F973068F534
:101630009093E900981739F07091EC002091ED003B
:101640005091F00003C0242F762F50E021FD02C0FE
:101650009F5FECCF3091EB003E7F3093EB003091F9
:10166000ED003D7F3093ED003091EB003160309321
:10167000EB007093EC002093ED005093F00020916C
:10168000EE0027FDE5CF80E008958F708093E9009C
:1016900081E008958091E50187FF11C08091E80005
:1016A00082FD05C08091E4018111F8CF11C08091C5
:1016B000E8008B770BC08091E401882349F080918A
:1016C000E80080FFF8CF8091E8008E778093E800F3
:1016D00008952091E4003091E50095E64091EC00FA
:1016E000842F817040FF23C08091E80080FD1DC0E1
:1016F0008091E401882399F0853099F08091EB0086
:1017000085FD11C04091E4005091E5002417350794
:1017100029F3915011F09A01E1CF84E0089582E01D
:10172000089583E0089581E0089580E00895409150
:10173000E80042FFDDCF08950E940A0C0E94120CBF
:10174000E0EEF0E0808181608083E8EDF0E0808170
:101750008F77808319BCA7EDB0E08C918E7F8C933E
:1017600080818F7E80831092E30108950F931F93F1
:10177000CF93DF930E940A0C0E94120CC8EDD0E0B8
:1017800088818F77888388818068888388818F7D2E
:10179000888319BC1092E4011092E0011092E201DA
:1017A0001092E10100EE10E0F80180818B7F8083D0
:1017B00088818160888342E060E080E00E94150BB0
:1017C000E1EEF0E080818E7F8083E2EEF0E08081C8
:1017D00081608083808188608083F80180818E7F32
:1017E0008083888180618883DF91CF911F910F91E1
:1017F0000895E8EDF0E080818F7E8083E7EDF0E0F2
:1018000080818160808384E082BF81E08093E301F6
:101810000C94B60BE8EDF0E080818E7F808310920F
:10182000E20008951092DA001092E10008951F92EC
:101830000F920FB60F9211242F933F934F935F9304
:101840006F937F938F939F93AF93BF93EF93FF9388
:101850008091E10082FF0BC08091E20082FF07C00F
:101860008091E1008B7F8093E1000E94830E809144
:10187000DA0080FF1FC08091D80080FF1BC08091DC
:10188000DA008E7F8093DA008091D90080FF0DC04E
:1018900080E189BD82E189BD09B400FEFDCF81E010
:1018A0008093E4010E947C0805C019BC1092E401F9
:1018B0000E948A088091E10080FF19C08091E200B7
:1018C00080FF15C08091E2008E7F8093E2008091BE
:1018D000E20080618093E2008091D8008062809372
:1018E000D80019BC85E08093E4010E948E088091A5
:1018F000E10084FF30C08091E20084FF2CC080E1D1
:1019000089BD82E189BD09B400FEFDCF8091D80078
:101910008F7D8093D8008091E1008F7E8093E100DD
:101920008091E2008F7E8093E2008091E2008160EE
:101930008093E2008091E001882311F084E007C0E9
:101940008091E30087FD02C081E001C083E08093C5
:10195000E4010E9490088091E10083FF29C08091FA
:10196000E20083FF25C08091E100877F8093E10042
:1019700082E08093E4011092E0018091E1008E7F8B
:101980008093E1008091E2008E7F8093E20080915D
:10199000E20080618093E20042E060E080E00E942B
:1019A000150B8091F00088608093F0000E948D08F4
:1019B000FF91EF91BF91AF919F918F917F916F9127
:1019C0005F914F913F912F910F900FBE0F901F90FD
:1019D00018951F920F920FB60F9211242F933F93D9
:1019E0004F935F936F937F938F939F93AF93BF9327
:1019F000CF93DF93EF93FF93C091E900CF70809175
:101A0000EC00D82FD17080FDD0E81092E9008091D1
:101A1000F000877F8093F00078940E942D0D109243
:101A2000E9008091F00088608093F000CD2BCF70AA
:101A3000C093E900FF91EF91DF91CF91BF91AF91FA
:101A40009F918F917F916F915F914F913F912F91D6
:101A50000F900FBE0F901F9018951F93CF93DF9399
:101A6000CDB7DEB7AA970FB6F894DEBF0FBECDBFD5
:101A7000E5EEF1E08091F100819321E0ED3EF20787
:101A8000C9F70E94AC088091E80083FF24C18091CF
:101A9000E5019091E601492F50E04A30510508F0E8
:101AA0001AC1FA01EA5AFF4F0C94E122803881F002
:101AB000823809F010C18091E9018F708093E900AC
:101AC0008091EB0085FB882780F91092E90006C021
:101AD0008091E1019091E201911182609091E80082
:101AE000977F9093E8008093F1001092F100C8C0B6
:101AF000282F2D7F09F0EFC0882319F0823061F084
:101B0000EAC08091E701813009F0E5C0933009F027
:101B100080E08093E2012BC08091E701811127C012
:101B20008091E9018F7009F4D6C08093E90020917B
:101B3000EB0020FF1CC0933021F48091EB00806209
:101B400014C09091EB0090619093EB0021E030E0A5
:101B5000A90102C0440F551F8A95E2F74093EA009D
:101B60001092EA008091EB0088608093EB00109265
:101B7000E9008091E800877F86C08111ACC0109198
:101B8000E7011F778091E3008078812B8093E30049
:101B90008091E800877F8093E8000E944A0B809143
:101BA000E80080FFFCCF8091E30080688093E30031
:101BB000111102C082E001C083E08093E4018BC078
:101BC0008058823008F087C08091E7019091E80149
:101BD0008C3D53E0950779F583E08A838AE2898317
:101BE0004FB7F894DE01139620E03EE051E2E32F78
:101BF000F0E050935700E49120FF03C0E295EF70AE
:101C00003F5FEF708E2F90E0EA3010F0C79601C072
:101C1000C0968D939D932F5F243149F74FBF8091DC
:101C2000E800877F8093E8006AE270E0CE010196C9
:101C30000E94560A14C0AE014F5F5F4F6091E901E8
:101C40000E949F09BC01892B09F445C09091E800CE
:101C5000977F9093E80089819A810E94B40A8091CD
:101C6000E8008B778093E80036C08038A1F580913A
:101C7000E800877F8093E8008091E0018093F10085
:101C80008091E8008E778093E8000E944A0B23C081
:101C9000811121C08091E7019091E8019927029775
:101CA000D4F48091E800877F8093E8008091E70179
:101CB0008093E0010E944A0B8091E001811106C0EF
:101CC0008091E30087FD02C081E001C084E0809341
:101CD000E4010E9498088091E80083FF0AC0809187
:101CE000E800877F8093E8008091EB00806280931A
:101CF000EB00AA960FB6F894DEBF0FBECDBFDF9102
:101D0000CF911F9108950895CF938091E401882386
:101D1000A1F0C091E900CF709091EC00892F817003
:101D200090FD80E8C82B1092E9008091E80083FDC7
:101D30000E942D0DCF70C093E900CF91089590932C
:101D40006901809368010895E0916801F09169014B
:101D5000309721F00190F081E02D099480E0089502
:101D6000E0916801F0916901309721F00280F381E0
:101D7000E02D09940895E0916801F0916901309790
:101D800021F00480F581E02D0994089520916601E9
:101D9000309167012817390771F09093670180939C
:101DA0006601E0916801F0916901309721F00680A9
:101DB000F781E02D09940895209164013091650127
:101DC0002817390771F09093650180936401E091C1
:101DD0006801F0916901309721F00084F185E02DD0
:101DE0000994089508950C94F20E0E94B01A0E946E
:101DF00062040C94761BCF92DF92EF92FF920F93C6
:101E00001F93CF93DF93CDB7DEB72B970FB6F89420
:101E1000DEBF0FBECDBF0E947A048BE6C82E81E0E4
:101E2000D82E00E010E0E02E802F0E947005F60111
:101E300041916F01F82EF426B1F40F5F1F4F0E3061
:101E4000110589F78FEF89838A831B820E94B91A53
:101E50008160782F9D838C8349815A816B818D812C
:101E60000E949E0F40C09091CC0191FF04C08B87CF
:101E70000E9476058B8520E030E04F2D50E0922FB8
:101E8000BA01022E02C0759567950A94E2F760FFC9
:101E900024C02E83EF8221E030E0690102C0CC0C27
:101EA000DD1C9A95E2F790E08C219D21892B09F4A5
:101EB00020E028870E94B91A8160782F9A87898745
:101EC0004E815F8168858A850E949E0FF801E559E1
:101ED000FE4F8081C826C08206C02F5F3F4F26304C
:101EE000310569F6AACF0E945D1E0E94A40E909152
:101EF0006A018917A1F00E94A40E80936A012B96B3
:101F00000FB6F894DEBF0FBECDBFDF91CF911F910A
:101F10000F91FF90EF90DF90CF900C949A072B9643
:101F20000FB6F894DEBF0FBECDBFDF91CF911F91EA
:101F30000F91FF90EF90DF90CF900895CF93DF93B4
:101F4000CDB7DEB72B970FB6F894DEBF0FBECDBF6F
:101F50004F83588769877A878B87DE01119686E0E1
:101F6000FD0111928A95E9F785E0FE01379601900F
:101F70000D928A95E1F749815A816B817C818D812F
:101F80009E810E94A1162B960FB6F894DEBF0FBE5D
:101F9000CDBFDF91CF910895CF93C82F882309F447
:101FA000C1C0823859F40E94A40E81FDBBC089E3F0
:101FB0000E943E190E94F61989E30CC0833879F417
:101FC0000E94A40E80FDAEC083E50E943E190E94CF
:101FD000F61983E50E947D19CF910C94F619843887
:101FE00059F40E94A40E82FD9DC087E40E943E1910
:101FF0000E94F61987E4EECF8CEF8C0F813A48F4FB
:102000008C2F0E949D2081118DC08C2F0E943E1923
:10201000E3CF80E28C0F883048F4C77081E001C0C4
:10202000880FCA95EAF70E94BF19D6CF8BE58C0FAF
:10203000833078F4C53A29F0C63A31F083E890E06D
:1020400005C081E890E002C082E890E0CF910C9456
:10205000C60E88E58C0F833108F064C0C83A39F1A8
:10206000C93A41F1CA3A49F1CB3A51F1CC3A59F166
:10207000CD3A61F1C03B69F1CE3A71F1CF3A79F1D5
:10208000C13B81F1C23B89F1C33B91F1C43B99F162
:10209000C53BA1F1C63BA9F1C73BB1F1C83BB9F1C2
:1020A000C93BC1F1CA3BC9F180E090E038C082EE83
:1020B00090E035C089EE90E032C08AEE90E02FC00B
:1020C00085EB90E02CC086EB90E029C087EB90E098
:1020D00026C08CEC90E023C08DEC90E020C083E81B
:1020E00091E01DC08AE891E01AC082E991E017C032
:1020F00084E991E014C081E292E011C083E292E0B1
:102100000EC084E292E00BC085E292E008C086E255
:1021100092E005C087E292E002C08AE292E0CF91AD
:102120000C94DC0ECF910895882309F44BC08238BB
:1021300059F40E94A40E81FF45C089E30E943E1914
:102140000E94F61989E30CC0833871F40E94A40E32
:1021500080FF38C083E50E943E190E94F61983E58E
:102160000E947D190C94F619843859F40E94A40E2B
:1021700082FF28C087E40E943E190E94F61987E476
:10218000EFCF9CEF980F913A58F390E2980F983068
:1021900050F4877091E001C0990F8A95EAF7892F72
:1021A0000E94C519DFCF9BE5980F933020F480E0A3
:1021B00090E00C94C60E885A833120F480E090E0C1
:1021C0000C94DC0E0895882321F00E94BF190C9412
:1021D000F6190895882321F00E94C5190C94F61968
:1021E0000895BF92CF92DF92EF92FF920F931F93C9
:1021F000CF93DF9300D000D000D0CDB7DEB77C0105
:1022000085E0F701DE01119601900D928A95E1F7C4
:10221000F70183819481892B09F4DDC2908181814A
:102220008F3F19F49F3F09F4D6C2F701028125813F
:1022300022952F7099838A8389819A812E830E94A7
:10224000FD18182FB92E0E94FC180E94C317EB2D01
:10225000E295EF704E2F50E0FA01E05AFF4F2E81C9
:102260000C94E1228B2D807F9B2D9F70F92E88236B
:1022700019F0F29480EFF822002349F0FF2009F4CE
:1022800057C28F2D0E94CF190E94F61951C2812F7B
:102290000E949410FF2009F49EC28F2D0E94D51930
:1022A00026960FB6F894DEBF0FBECDBFDF91CF915B
:1022B0001F910F91FF90EF90DF90CF90BF900C9403
:1022C000F6193B2D307F8B2D8F70303211F08295B7
:1022D000807F112319F0113021F12CC00023B9F0B7
:1022E000222309F490C1213009F08DC126960FB642
:1022F000F894DEBF0FBECDBFDF91CF911F910F913C
:10230000FF90EF90DF90CF90BF900C94DF192223C5
:1023100019F0213009F45FC28E830E94E2198E8188
:1023200086C1002321F0223008F055C26CC1211172
:1023300052C27DC1002321F0222309F464C1F8C1F7
:10234000222309F474C109C28B2D8695869583706A
:1023500019F08130D1F03FC2002321F0812F9B2D55
:10236000937002C080E090E026960FB6F894DEBF2E
:102370000FBECDBFDF91CF911F910F91FF90EF90D6
:10238000DF90CF90BF900C94C60E002321F0812FD8
:102390009B2D937002C080E090E026960FB6F894D3
:1023A000DEBF0FBECDBFDF91CF911F910F91FF9088
:1023B000EF90DF90CF90BF900C94DC0E812F002324
:1023C00019F00E94651D02C00E94CD1D26960FB611
:1023D000F894DEBF0FBECDBFDF91CF911F910F915B
:1023E000FF90EF90DF90CF90BF900C94521E8B2DFA
:1023F000837009F075C00111EEC1812F8295869519
:102400008770880F880F912F9F70C92ED12CE12CD7
:10241000F12C082E04C0CC0CDD1CEE1CFF1C0A9411
:10242000D2F714FF12C00FE010E020E030E004C04B
:10243000000F111F221F331F8A95D2F7C901B8015F
:10244000609570958095909503C060E070E0CB0139
:102450004B2D4695469543704230C1F060F56C298E
:102460007D298E299F29413051F126960FB6F89487
:10247000DEBF0FBECDBFDF91CF911F910F91FF90B7
:10248000EF90DF90CF90BF900C94EA176C297D29D4
:102490008E299F2926960FB6F894DEBF0FBECDBFBA
:1024A000DF91CF911F910F91FF90EF90DF90CF9030
:1024B000BF900C9406180E94EA17C701B601269631
:1024C0000FB6F894DEBF0FBECDBFDF91CF911F9145
:1024D0000F91FF90EF90DF90CF90BF900C94CE17AC
:1024E000002319F08B2D817001C08695882309F493
:1024F00072C1812F829586958770880F880F912FE2
:102500009F70C92ED12CE12CF12C082E04C0CC0CCC
:10251000DD1CEE1CFF1C0A94D2F714FF12C00FE062
:1025200010E020E030E004C0000F111F221F331F15
:102530008A95D2F7C901B8016095709580959095FC
:1025400003C060E070E0CB014B2D4695469543708B
:102550004230C1F060F56C297D298E299F294130D8
:1025600051F126960FB6F894DEBF0FBECDBFDF91B6
:10257000CF911F910F91FF90EF90DF90CF90BF9080
:102580000C94C4186C297D298E299F2926960FB694
:10259000F894DEBF0FBECDBFDF91CF911F910F9199
:1025A000FF90EF90DF90CF90BF900C94E0180E94C6
:1025B000C418C701B60126960FB6F894DEBF0FBE49
:1025C000CDBFDF91CF911F910F91FF90EF90DF90E2
:1025D000CF90BF900C94A818103FD1F118F4103E82
:1025E00050F4A1C0123F09F463C008F44CC0133F7B
:1025F00009F473C098C01F708B2D8F710023A1F058
:102600000E944118812F26960FB6F894DEBF0FBEA8
:10261000CDBFDF91CF911F910F91FF90EF90DF9091
:10262000CF90BF900C94E3100E946218812F2696E1
:102630000FB6F894DEBF0FBECDBFDF91CF911F91D3
:102640000F91FF90EF90DF90CF90BF900C94EA1025
:102650000023A9F02111BFC08B2D8F7126960FB6D4
:10266000F894DEBF0FBECDBFDF91CF911F910F91C8
:10267000FF90EF90DF90CF90BF900C94871822309E
:1026800008F0A9C0E9CF0023A9F08B2D8F71269601
:102690000FB6F894DEBF0FBECDBFDF91CF911F9173
:1026A0000F91FF90EF90DF90CF90BF900C94411866
:1026B000002359F38B2D8F7126960FB6F894DEBF49
:1026C0000FBECDBFDF91CF911F910F91FF90EF9083
:1026D000DF90CF90BF900C946218002399F08B2D5F
:1026E0008F7126960FB6F894DEBF0FBECDBFDF9177
:1026F000CF911F910F91FF90EF90DF90CF90BF90FF
:102700000C942C1826960FB6F894DEBF0FBECDBFE2
:10271000DF91CF911F910F91FF90EF90DF90CF90BD
:10272000BF900C9422180023A9F0222309F4ADCF06
:10273000812F26960FB6F894DEBF0FBECDBFDF9176
:10274000CF911F910F91FF90EF90DF90CF90BF90AE
:102750000C94CC0F222309F4ADCF812F26960FB60F
:10276000F894DEBF0FBECDBFDF91CF911F910F91C7
:10277000FF90EF90DF90CF90BF900C9494104B2D72
:102780004F70612FC7010E94020326960FB6F8947E
:10279000DEBF0FBECDBFDF91CF911F910F91FF9094
:1027A000EF90DF90CF90BF900C9446174B2D4F7059
:1027B000612FC70126960FB6F894DEBF0FBECDBFBE
:1027C000DF91CF911F910F91FF90EF90DF90CF900D
:1027D000BF900C94370626960FB6F894DEBF0FBE56
:1027E000CDBFDF91CF911F910F91FF90EF90DF90C0
:1027F000CF90BF9008950E94DC190E94B1190E94E9
:10280000F6190E94021F0E94521E80E090E00E9472
:10281000C60E80E090E00C94DC0E0E94CC190C9463
:10282000FB130E94FD18292F22952F702C3030F4B5
:102830002A3048F42250223078F405C02C3041F080
:102840002F3031F009C0803E48F0803F29F406C0A7
:1028500093FB882780F9089580E0089581E008952A
:10286000CF93DF9300D000D01F92CDB7DEB70F908B
:102870000F900F900F900F90DF91CF910895CF930D
:10288000DF9300D000D000D0CDB7DEB726960FB6CC
:10289000F894DEBF0FBECDBFDF91CF9108951F9397
:1028A000CF93DF93C091790116E080917A01C81728
:1028B00099F0D0E01C9FF0011D9FF00D1124E55808
:1028C000FE4F4081518162817381848195810E9494
:1028D0003F142196C770E9CFDF91CF911F910895E2
:1028E0004091AB015091AC016091AD017091AE018E
:1028F0008091AF019091B0010C943F148091B00190
:1029000082958F7009F054C08091AD01882309F43D
:102910004FC080917901A0917A014091AE01509110
:10292000AF016091AB017091AC01B6E08A1709F478
:102930003FC090E041155105C1F17F3F11F46F3F59
:10294000A1F1B89FF001B99FF00D1124E558FE4F99
:10295000218127132AC02081261327C0228121111B
:1029600024C0238134812417350710F42150310904
:10297000241B350B283C3105C0F42091B0012F7089
:1029800020612093B00126E0289FF001299FF00DDF
:102990001124E058FE4F80818F70806180838BEA24
:1029A00091E00E94F1100C944F1401968770BECFF5
:1029B0000895CF92DF92EF92FF920F931F93CF93E0
:1029C000DF93CDB7DEB762970FB6F894DEBF0FBEC8
:1029D000CDBF8C0185E0F801DE011D9601900D92BE
:1029E0008A95E1F7D8014C9111965C911197129656
:1029F0006C918091AE019091AF01009709F475C17F
:102A00003091AB017091AC017F3F19F43F3F09F465
:102A10006CC1F801C380D480E090AD01EE2009F4D0
:102A2000BEC02091B001C816D90628F0D601A81B57
:102A3000B90BCD0104C0809590958C0D9D1DFF2490
:102A4000F394883C910578F0F12C207F09F0C4C004
:102A50007C2DD98AC88A89890E9430148BEA91E03A
:102A60000E94F110AFC0822F807F09F045C057133C
:102A700013C0431311C061110FC02F702061209348
:102A8000B0010E9470148BEA91E00E94F1108091D5
:102A9000B001F80185832EC0CD2819F15F3F11F4F4
:102AA0004F3FF9F0F62E61111CC080917901209101
:102AB0007A0136E0821709F45BC090E0389FF0019C
:102AC000399FF00D1124E558FE4F7181571306C050
:102AD0007081471303C07281711103C00196877022
:102AE000E9CFF62E662309F41CC18091B001816004
:102AF0008093B001F12C15C1571309C0431307C0CF
:102B0000611105C08091B001F8018583C8C04D876F
:102B10005E878D859E856A8B0E9411146A89882341
:102B2000D1F16623C1F12091B001822F82958F707F
:102B300090E0029774F08091AB019091AC0198877E
:102B40008F831986DB86CA862C87CE0107960E9462
:102B5000F11086E0F801ABEAB1E001900D928A95A0
:102B6000E1F70E947E140E947014FF24F394D9C0F0
:102B70004D875E878D859E850E94FD18292F2295A1
:102B80002F70223008F0C1C09F7009F0BBC0805E7A
:102B9000883008F4C6C0C8010E94F110E6CFC816FC
:102BA000D90608F453C0F601E81BF90BCF01883CA5
:102BB000910508F450C0F12C7C2DD98AC88A8989E6
:102BC0000E943014EBEAF1E086E0DF011D928A9565
:102BD000E9F70E947014A5C0571314C0431312C024
:102BE000611110C08091B001F8018583C8010E9475
:102BF000F11086E0EBEAF1E0DF011D928A95E9F73A
:102C0000FE2C8FC04D875E878D859E856A8B0E94C6
:102C100011146A89882309F4BECF662309F4BBCF57
:102C20002091B001822F82958F7090E002970CF472
:102C300090CF8091AB019091AC019A8389831B82E4
:102C4000DD82CC822E83CE01019681CF8095909536
:102C50008C0D9D1DACCFF62E662309F49CCF571327
:102C600033C0431331C02091B00120FD24C0822F16
:102C700082958F70482F50E041155105E1F0D80141
:102C800015962C9315974F30510549F08F5F982F6B
:102C90009295907F822F8F70892B15968C93C80107
:102CA0000E94F11086E0F801ABEAB1E001900D92CC
:102CB0008A95E1F78ECF86E0F801ABEAB1E00190AA
:102CC0000D928A95E1F72DC04D875E878D859E8593
:102CD0000E94111481113DCF8091B00181608093D9
:102CE000B001C8010E94F1101CC0662309F453CF43
:102CF0004D875E878D859E850E941114882309F477
:102D00004ACF27CF811143CF0CC0243008F043CFE6
:102D10009F7009F43CCFD80115969C91907F09F0E3
:102D200036CF8F2D62960FB6F894DEBF0FBECDBFA3
:102D3000DF91CF911F910F91FF90EF90DF90CF9097
:102D400008951F93CF93DF93CDB7DEB72C970FB6BF
:102D5000F894DEBF0FBECDBF4F83588769877A874F
:102D60008B879C87CE0107960E94D914882371F027
:102D70008A859B85892B09F441C088858F3F09F09E
:102D800065C08F818F3F09F061C038C086E0FE01C9
:102D90003796DE01119601900D928A95E1F76A85CA
:102DA0007B856115710551F1FF81E885EF3F11F4D5
:102DB000FF3F21F120917A0130E0C901019687702F
:102DC00099274091790150E08417950709F447C08D
:102DD000F983EA837D836C8396E0929FD001939F71
:102DE000B00D1124A558BE4FFE01319601900D92F1
:102DF0009A95E1F780937A010E944F1416E0809132
:102E0000790190917A018917B9F1189FC0011124B5
:102E100085589E4F0E94D914882371F1E091790161
:102E20001E9FF0011124E558FE4F408151816281BF
:102E30007381848195810E943F148091790190E093
:102E400001968770992780937901D9CF4F81588552
:102E500069857A858B859C850E943F14CFCF0E941F
:102E60000D1410927A0110927901EBEAF1E086E0FC
:102E7000DF011D928A95E9F72C960FB6F894DEBF14
:102E80000FBECDBFDF91CF911F910895EF92FF92BA
:102E90000F931F93CF93DF938C01892B09F46CC0A0
:102EA000F12CEE24E394E8012196F8018491843713
:102EB00040F4843008F051C0813081F0823019F143
:102EC0005BC0853709F444C0A8F19CE7980F9037A0
:102ED00008F052C08F770E94941041C00E5F1F4FC0
:102EE000FE01849190E2980F983050F48770FE2D87
:102EF00001C0FF0F8A95EAF78F2F0E94CF1914C0E7
:102F00000E94CC0F2DC00E5F1F4FFE01849190E2F6
:102F1000980F983060F48770FE2D01C0FF0F8A95DE
:102F2000EAF78F2F0E94D5190E94F61919C00E9446
:102F3000941016C00E5F1F4FFE01C491CC2381F088
:102F40008FE99FE00197F1F700C00000C150F6CF74
:102F50000E5F1F4FFE01F49003C00E94CC0F8E0144
:102F60008F2D882309F49FCFEFE9FFE03197F1F728
:102F700000C000008150F5CFDF91CF911F910F91DC
:102F8000FF90EF90089508956093B5017093B60196
:102F90008093B7019093B8010C94FB130F931F9388
:102FA0000091B5011091B6012091B7013091B8019F
:102FB000DC01CB01802B912BA22BB32B8093B5018D
:102FC0009093B601A093B701B093B8011F910F91F0
:102FD0000C94FB130F931F930091B5011091B60150
:102FE0002091B7013091B801DC01CB0180239123FE
:102FF000A223B3238093B5019093B601A093B701A8
:10300000B093B8011F910F910C94FB130F931F9372
:103010000091B5011091B6012091B7013091B8012E
:10302000DC01CB0180279127A227B3278093B5012C
:103030009093B601A093B701B093B8011F910F917F
:103040000C94FB131092B1011092B2011092B301D3
:103050001092B4010C94FB1341E050E060E070E08A
:1030600004C0440F551F661F771F8A95D2F74093FF
:10307000B1015093B2016093B3017093B4010C9409
:10308000FB1341E050E060E070E004C0440F551FC6
:10309000661F771F8A95D2F78091B1019091B20196
:1030A000A091B301B091B401482B592B6A2B7B2B13
:1030B0004093B1015093B2016093B3017093B40196
:1030C0000C94FB1341E050E060E070E004C0440F5A
:1030D000551F661F771F8A95D2F7409550956095CA
:1030E00070958091B1019091B201A091B301B0911E
:1030F000B401482359236A237B234093B1015093A1
:10310000B2016093B3017093B4010C94FB1341E0DE
:1031100050E060E070E004C0440F551F661F771F49
:103120008A95D2F78091B1019091B201A091B3013B
:10313000B091B401482759276A277B274093B101F2
:103140005093B2016093B3017093B4010C94FB13DC
:103150000F931F930091B1011091B2012091B3011F
:103160003091B401DC01CB01802B912BA22BB32B2E
:103170008093B1019093B201A093B301B093B401D5
:103180001F910F910C94FB130F931F930091B101AA
:103190001091B2012091B3013091B401DC01CB0157
:1031A00080239123A223B3238093B1019093B20192
:1031B000A093B301B093B4011F910F910C94FB1332
:1031C0000F931F930091B1011091B2012091B301AF
:1031D0003091B401DC01CB0180279127A227B327CE
:1031E0008093B1019093B201A093B301B093B40165
:1031F0001F910F910C94FB130895CF92DF92EF92E1
:10320000FF920F931F93CF93DF938C01C090B10176
:10321000D090B201E090B301F090B4018091B5017B
:103220009091B601A091B701B091B801C82AD92AEE
:10323000EA2AFB2ACFE1D0E0D701C6010C2E04C058
:10324000B695A795979587950A94D2F780FF07C002
:10325000B8018C2F0E945B068130910531F42197D3
:1032600058F7B80180E00E945B06DF91CF911F9173
:103270000F91FF90EF90DF90CF90089590910C0107
:103280009923F1F090910D019923D1F0982F969503
:10329000969596959F3080F5E0910E01F0910F0183
:1032A000E90FF11D877021E030E0A90102C0440F51
:1032B000551F8A95E2F7CA019181892B8183089570
:1032C00020910E0130910F01F90132969FEF40E0FD
:1032D0005191851789F09F3F19F4511101C0942F26
:1032E0004F5F4E30A9F79F3F39F0F901E90FF11D0B
:1032F00097FDFA9582830895089590910C01992382
:10330000F9F090910D019923D9F0982F9695969503
:1033100096959F3028F5E0910E01F0910F01E90F8D
:10332000F11D877021E030E0A90102C0440F551F54
:103330008A95E2F7CA018095918189238183089556
:1033400020910E0130910F01F9013296205F3F4F1D
:103350009081891301C010823196E217F307C1F7FB
:10336000089581E090E0E0910E01F0910F01E80FE7
:10337000F91F1082019680319105A9F70895909167
:10338000CB01892B8093CB01089580959091CB013F
:1033900089238093CB0108951092CB0108959091D9
:1033A000CA01892B8093CA01089580959091CA0122
:1033B00089238093CA0108951092CA0108958093C9
:1033C000B90108951092B901089580910E0190916C
:1033D0000F01FC0131969C01205F3F4F80E09191ED
:1033E00091118F5FE217F307D1F70895E0910E0175
:1033F000F0910F018091CB018083E0910E01F0915B
:103400000F0190818091CA01892B80838091B9013D
:10341000882361F0E0910E01F0910F019081892BDA
:1034200080830E94E51981111092B90180910E01EB
:1034300090910F010C94B00ECF92DF92EF92FF9219
:103440006C01EE24FF24C114D104E104F10421F045
:10345000C701B60120E101C020E0C72ED82EE92E19
:10346000FF24C114D104E104F10419F0285FC7015D
:10347000B6016B017C0154E0F694E794D794C794AD
:103480005A95D1F7C114D104E104F10419F02C5F6D
:10349000C701B6016B017C0142E0F694E794D79432
:1034A000C7944A95D1F7C114D104E104F10419F08D
:1034B0002E5FC701B601DC01CB01B695A7959795A4
:1034C0008795892B8A2B8B2B09F02F5F822FFF90FA
:1034D000EF90DF90CF9008958091E401843011F156
:1034E00020E488E190E00FB6F894A89580936000FE
:1034F0000FBE2093600083B7817F846083BF83B752
:10350000816083BF7894889583B78E7F83BF0FB621
:10351000F894A89580916000886180936000109273
:1035200060000FBE089508950C94931ACF930E94E3
:10353000941A0E947A040E94931AC0E08C2F0E9471
:103540007005811104C0CF5FCE30C1F701C081E0AA
:10355000CF9108950E940D140E94A40E0C949A0716
:1035600082E084BD93E095BD9AEF97BD80936E0095
:1035700008952FB7F8948091CD019091CE01A0913C
:10358000CF01B091D0012FBF0895CF92DF92EF927B
:10359000FF920F931F932FB7F8944091CD01509154
:1035A000CE016091CF017091D0012FBF6A017B01E4
:1035B000EE24FF248C0120E030E0C016D106E206A4
:1035C000F30610F4415051099A01281B390BC90127
:1035D0001F910F91FF90EF90DF90CF9008951F9271
:1035E0000F920FB60F9211248F939F93AF93BF93B7
:1035F0008091CD019091CE01A091CF01B091D001E9
:103600000196A11DB11D8093CD019093CE01A09391
:10361000CF01B093D001BF91AF919F918F910F9047
:103620000FBE0F901F9018950E949C0BF8942FEFDF
:1036300087EA91E6215080409040E1F700C0000009
:1036400087E090EBDC018093ED019093EE01A09375
:10365000EF01B093F0019CE088E10FB6F894A895D3
:10366000809360000FBE90936000FFCFEF92FF92B7
:103670000F931F93CF93DF93D82FC0E08C2F0E941E
:10368000700500E010E0E82EF12CC701002E02C00A
:10369000959587950A94E2F780FD06C00F5F1F4F4E
:1036A0000630110591F709C0602F7C2F80E00E9441
:1036B00038068D13F3CF81E004C0CF5FCE30F1F632
:1036C00080E0DF91CF911F910F91FF90EF900895CF
:1036D000CF93C82F8CE20E94361B882321F08C2FB9
:1036E000CF910C94361B80E0CF910895CF930E9428
:1036F000BD1C811102C00E94A31CC5E6C15049F047
:103700000E947A048FE39CE90197F1F700C0000062
:10371000F5CF89E20E94681B811113C18AE20E94E1
:10372000681B81110E94A31C85E00E94681B811107
:103730000E94141B0E94C81C8093CC0187E00E9449
:10374000681B8823A9F18BE10E94681B882351F034
:103750008091CC0181FB222720F991E0922790FBF8
:1037600081F90EC08EE00E94681B882361F0809171
:10377000CC0182FB222720F991E0922790FB82F96D
:103780008093CC0115C080E10E94681B9091CC0110
:10379000882341F093FB222720F981E0822780FBD8
:1037A00093F904C0892F809580FB90F99093CC0108
:1037B0008091CC010E94CC1C0E94DA1C8093DE0117
:1037C00080EE0E94681B882341F08091DE01982FD3
:1037D000909590FB80F98093DE0189E30E94681B3D
:1037E000882359F08091DE0181FB222720F991E0A6
:1037F000922790FB81F98093DE0182EE0E94681B84
:10380000882359F08091DE0182FB222720F991E084
:10381000922790FB82F98093DE0186EE0E94681B5E
:10382000882359F08091DE0183FB222720F991E063
:10383000922790FB83F98093DE0183EE0E94681B40
:10384000882359F08091DE0184FB222720F991E042
:10385000922790FB84F98093DE0185E30E94681B28
:10386000882359F08091DE0185FB222720F991E021
:10387000922790FB85F98093DE0181E30E94681B0B
:10388000882359F08091DE0186FB222720F991E000
:10389000922790FB86F98093DE0181E10E94681BEC
:1038A000882359F08091DE0187FB222720F991E0DF
:1038B000922790FB87F98093DE018091DE010E94C0
:1038C000DE1C8091DE0187FB882780F980930D0143
:1038D00087E20E94681BC82F8EE10E94681B81113D
:1038E000C2608FE10E94681B8111C46080E20E9467
:1038F000681B8111C86081E20E94681B8111C06150
:1039000082E20E94681B8111C06283E20E94681BF0
:103910008111C06484E20E94681B882311F0C06892
:1039200002C0CC2329F08C2F0E94D51C6C2F03C021
:103930000E94D11C682F70E080E090E0CF910C9441
:10394000C417CF9108956DEE7EEF80E090E00E9465
:10395000172360E082E090E00E94092360E083E0AA
:1039600090E00E94092360E084E090E00E94092337
:1039700060E085E090E00C94092380E090E00E94F4
:10398000032321E08D3E9E4F09F020E0822F089511
:1039900082E090E00C94FB22682F82E090E00C948F
:1039A000092383E090E00C94FB22682F83E090E0F1
:1039B0000C94092384E090E00C94FB22682F84E0AF
:1039C00090E00C9409238091D30180FF0BC060919B
:1039D000130185E0689FB001112475956795759571
:1039E00067952BC081FF09C06091130185E0689F36
:1039F000B00111247595679520C082FF07C06091C2
:103A0000130185E0689FB001112417C09091D40183
:103A10009923D1F060911201961788F72091130134
:103A200085E0289F90011124929FA001939F500D43
:103A3000112470E0CA010E94CD226038710540F463
:103A40006115710519F406C065E070E0862F0895D0
:103A50008FE7089581E008958091D30180FF08C029
:103A60006091110170E0759567957595679521C016
:103A700081FF06C06091110170E07595679519C0CE
:103A800082FF04C06091110170E010C09091D401D8
:103A9000992399F0609110019617A0F78091110178
:103AA000899FC001112470E00E94CD226038710509
:103AB00040F46115710519F406C061E070E0862FCD
:103AC00008958FE7089581E00895803F21F40E94D2
:103AD000E31C819504C0813F29F40E94E31C80937C
:103AE000D7010895823F21F40E94E31C819504C010
:103AF000833F29F40E94E31C8093D6010895893FF7
:103B000019F40E942C1D05C08A3F31F40E942C1D1F
:103B100081958093D80108958B3F21F40E942C1D3C
:103B2000819504C08C3F29F40E942C1D8093D901FB
:103B30000895843F21F48091D501816017C0853FAD
:103B400021F48091D501826011C0863F21F48091DB
:103B5000D50184600BC0873F21F48091D501886036
:103B600005C0883F31F48091D50180618093D501F3
:103B700008958D3F21F48091D30181600BC08E3F69
:103B800021F48091D301826005C08F3F29F4809198
:103B9000D30184608093D3010895803F39F48091EC
:103BA000D70187FF6CC01092D70169C0813F29F40B
:103BB0008091D7011816BCF362C09091D601823F64
:103BC00029F497FF5CC01092D60159C0833F19F4C5
:103BD0001916CCF354C0893F41F48091D8011816CE
:103BE0000CF04DC01092D8014AC08A3F29F4809150
:103BF000D80187FF44C0F6CF8B3F39F48091D901BB
:103C000087FF3DC01092D9013AC08C3F29F48091C2
:103C1000D9011816BCF333C0843F21F48091D5013B
:103C20008E7F17C0853F21F48091D5018D7F11C013
:103C3000863F21F48091D5018B7F0BC0873F21F413
:103C40008091D501877F05C0883F31F48091D501EF
:103C50008F7E8093D50113C08D3F21F48091D301D5
:103C60008E7F0BC08E3F21F48091D3018D7F05C0E4
:103C70008F3F29F48091D3018B7F8093D301809172
:103C8000D60181110EC08091D70181110AC08091A7
:103C9000D801811106C08091D901811102C0109212
:103CA000D401089585ED91E00E94BB0E0E94B91ADF
:103CB0009093D2018093D10108951F93CF93DF9306
:103CC0008091D1019091D2010E94C51AAC019091CE
:103CD000D401992321F02091140130E006C02091F5
:103CE00015018AE0289F900111244217530708F418
:103CF00085C08091D601C091D701D091D801109193
:103D0000D901811107C0C11175C0D11173C0111142
:103D100071C074C09F3F19F09F5F9093D401181633
:103D200024F40E94E31C8093D6018091D60187FF82
:103D300005C00E94E31C81958093D6011C1624F4D3
:103D40000E94E31C8093D7018091D70187FF05C0B3
:103D50000E94E31C81958093D7016091D601662370
:103D600031F1C091D701CC2311F1062E000C770B55
:103D7000880B990B0E94D42123E333E343E35FE3F1
:103D80000E9438220E949C216093D6016C2FCC0F98
:103D9000770B880B990B0E94D42123E333E343E391
:103DA0005FE30E9438220E949C216093D7011D1678
:103DB00024F40E942C1D8093D8018091D80187FFA4
:103DC00005C00E942C1D81958093D801111624F402
:103DD0000E942C1D8093D9018091D90187FF05C0D5
:103DE0000E942C1D81958093D901DF91CF911F9165
:103DF0000C94521E9F3F09F08FCFA0CFDF91CF913F
:103E00001F910895E5EDF1E085E0DF011D928A95AF
:103E1000E9F71092D4011092D3010895833081F113
:103E200028F4813059F08230D1F00895853009F4BA
:103E300049C0B8F1863009F456C008958091150143
:103E4000262F30E0280F311D2F3F310524F4680F55
:103E50006093150108958FEF809315010895809167
:103E60001401262F30E0280F311D2F3F310524F497
:103E7000680F6093140108958FEF809314010895E3
:103E800080911301262F30E0280F311D2F3F31057F
:103E900024F4680F6093130108958FEF809313014A
:103EA000089580911201262F30E0280F311D2F3FF9
:103EB000310524F4680F6093120108958FEF809309
:103EC0001201089580911101262F30E0280F311D35
:103ED0002F3F310524F4680F6093110108958FEF8F
:103EE00080931101089580911001262F30E0280F52
:103EF000311D2F3F310524F4680F609310010895A0
:103F00008FEF809310010895833011F128F48130F0
:103F100049F0823091F00895853081F120F18630AA
:103F2000C1F1089580911501681720F4861B8093D4
:103F300015010895109215010895809114016817D4
:103F400020F4861B809314010895109214010895A3
:103F500080911301681720F4861B80931301089544
:103F600010921301089580911201681720F4861BA6
:103F70008093120108951092120108958091110109
:103F8000681720F4861B8093110108951092110187
:103F9000089580911001681720F4861B809310010A
:103FA00008951092100108950F931F938D3109F415
:103FB0006BC008F03FC08E3009F47DC0C0F487307C
:103FC00009F46EC068F4863009F0AFC08091CC016E
:103FD000817F8E7F8093CC0181E08093DB01A6C03E
:103FE000883009F458C08B3009F49BC09EC08631DC
:103FF00009F497C078F4803109F470C0813109F078
:1040000094C00E940D1490910D0181E08927809346
:104010000D0187C0893109F484C08B3109F085C056
:104020008091CC0181FB222720F991E0922790FB1F
:1040300081F94AC0853309F45BC048F4873209F43A
:1040400057C008F45AC0893209F452C06EC0833494
:1040500038F48A3308F067C0883309F462C065C059
:10406000833409F445C0883409F05FC00E940D1400
:104070000FEF13ED20E3015010402040E1F700C0A6
:1040800000000E94141B4DC00E9456210E94A40EE5
:104090000E949A0746C00E94C81C0E94DA1C41C0B8
:1040A0009091CC01892F817090FF12C0917F9E7FEB
:1040B0009093CC013BC08091CC0182FB222720F958
:1040C00091E0922790FB82F98093CC01992349F1EA
:1040D0008091CC0181608093CC0123C08091CC0180
:1040E00083FB222720F991E0922790FB83F9ECCF04
:1040F00061E070E080E090E010C08D5141E050E060
:1041000060E070E08A019B0104C0000F111F221FB4
:10411000331F8A95D2F7C901B8010E94C4170E94C3
:104120000D1481E003C08953E9CF80E01F910F9106
:10413000089580E008950C949920CF93C82F809122
:10414000DB01813079F018F08230E9F187C0E0912D
:104150000E01F0910F018081813169F0823209F006
:104160007FC009C0E0910E01F0910F018081813183
:1041700011F0823261F48C2F0E949B20811104C0C7
:104180008C2F0E94D41F1DC081E090E01AC08C2F9C
:104190000E949920811114C0C43179F048F4CB30C9
:1041A00079F0C03109F060C082E08093DB0108C083
:1041B000C93219F0C83321F057C01092DB0154C046
:1041C00081E0817053C0C93289F118F5C43171F1B1
:1041D000A8F4C73009F046C08AE08093150194E145
:1041E0009093140193E0909313018093120188E05F
:1041F0008093110188E28093100134C0CE51C63003
:1042000088F5EC2FF0E0E65DFE4F80818093DA01C7
:1042100029C0CE34E9F020F4CB3421F56AE013C094
:10422000C13579F0C235F1F461E00DC08091DA0159
:10423000882319F01092DA0115C081E08093DB0128
:1042400015C061E006C08091DA010E940E1F0AC00D
:104250006AE08091DA010E94841F04C01092DB01A1
:1042600080E004C081E002C080E0ABCFCF91089530
:10427000E1E8F0E0808188608083808181608083D4
:104280008FB7F89493E09093890090ED9093880015
:104290008FBF0895EFE6F0E080818260808308950B
:1042A000EFE6F0E080818D7F80830895EFE6F0E017
:1042B000908182E08927808308951F920F920FB624
:1042C0000F9211242F933F934F935F936F937F939C
:1042D0008F939F93AF93BF93EF93FF938091DC01F4
:1042E0009091DD0101969093DD018093DC018111B5
:1042F00003C082E00E949A07E091DD01E695E69511
:10430000F0E0EE5CFA4FE4918091DC018E1303C083
:1043100080E00E949A07FF91EF91BF91AF919F912A
:104320008F917F916F915F914F913F912F910F905E
:104330000FBE0F901F9018950E94A3216894B11191
:104340000C94322208950E94172288F09F5798F00B
:10435000B92F9927B751B0F0E1F0660F771F881F8A
:10436000991F1AF0BA95C9F714C0B13091F00E94A4
:104370003122B1E008950C943122672F782F8827DD
:10438000B85F39F0B93FCCF3869577956795B395CB
:10439000D9F73EF490958095709561957F4F8F4F3A
:1043A0009F4F0895E89409C097FB3EF4909580953F
:1043B000709561957F4F8F4F9F4F9923A9F0F92FEB
:1043C00096E9BB279395F695879577956795B79569
:1043D000F111F8CFFAF4BB0F11F460FF1BC06F5F4F
:1043E0007F4F8F4F9F4F16C0882311F096E911C061
:1043F000772321F09EE8872F762F05C0662371F082
:1044000096E8862F70E060E02AF09A95660F771F95
:10441000881FDAF7880F9695879597F9089557FDC5
:104420009058440F551F59F05F3F71F04795880F22
:1044300097FB991F61F09F3F79F0879508951216B9
:1044400013061406551FF2CF4695F1DF08C0161665
:1044500017061806991FF1CF869571056105089416
:104460000895E894BB2766277727CB0197F908952D
:104470000E944B220C94BC220E94AE2238F00E9473
:10448000B52220F0952311F00C94A5220C94AB22B8
:1044900011240C9432220E940F2270F3959FC1F3D5
:1044A000950F50E0551F629FF001729FBB27F00DE2
:1044B000B11D639FAA27F00DB11DAA1F649F662737
:1044C000B00DA11D661F829F2227B00DA11D621F86
:1044D000739FB00DA11D621F839FA00D611D221F40
:1044E000749F3327A00D611D231F849F600D211D24
:1044F000822F762F6A2F11249F5750409AF0F1F0A7
:1045000088234AF0EE0FFF1FBB1F661F771F881F0F
:1045100091505040A9F79E3F510580F00C94A52280
:104520000C9432225F3FE4F3983ED4F3869577955E
:104530006795B795F795E7959F5FC1F7FE2B880FB5
:10454000911D9695879597F9089597F99F6780E84B
:1045500070E060E008959FEF80EC089500240A94D5
:104560001616170618060906089500240A9412164E
:104570001306140605060895092E0394000C11F481
:10458000882352F0BB0F40F4BF2B11F460FF04C02E
:104590006F5F7F4F8F4F9F4F089597FB072E16F445
:1045A000009407D077FD09D00E94E72207FC05D0D0
:1045B0003EF4909581959F4F0895709561957F4F3A
:1045C0000895EE0FFF1F0590F491E02D0994AA1BAA
:1045D000BB1B51E107C0AA1FBB1FA617B70710F0EE
:1045E000A61BB70B881F991F5A95A9F78095909520
:1045F000BC01CD010895F999FECF92BD81BDF89A15
:10460000992780B50895A8E1B0E042E050E00C940D
:104610001E23262FF999FECF1FBA92BD81BD20BD62
:104620000FB6F894FA9AF99A0FBE019608950E946F
:104630000923272F0C940A23DC01CB01FC01F999F3
:10464000FECF06C0F2BDE1BDF89A319600B40D92DE
:0C46500041505040B8F70895F894FFCF97
:10465C0020029B072B080608D2079E070101BA010E
:10466C0028080A03140A3F4D3639F304A6047004D3
:10467C003704CA03E303FC03150401020304050613
:04468C000708090012
:00000001FF
